S02200006F70656E626C745F6E75636C656F5F73746D33326631303372622E7372656343
S315080000000050002075160008BD160008BD16000829
S31508000010BD160008BD160008BD1600080000000041
S31508000020000000000000000000000000BD160008E7
S31508000030BD16000800000000BD1600088D05000862
S31508000040BD160008BD160008BD160008BD16000836
S31508000050BD160008BD160008BD160008BD16000826
S31508000060BD160008BD160008BD160008BD16000816
S31508000070BD160008BD160008BD160008BD16000806
S31508000080BD160008BD160008BD160008BD160008F6
S31508000090BD160008BD160008BD160008BD160008E6
S315080000A0BD160008BD160008BD160008BD160008D6
S315080000B0BD160008BD160008BD160008BD160008C6
S315080000C0BD160008BD160008BD160008BD160008B6
S315080000D0BD160008BD160008BD160008BD160008A6
S315080000E0BD160008BD160008BD1600080000000071
S315080000F000000000000000000000000000000000F2
S3110800010000000000000000005FF808F195
S3150800010C10B5054C237833B9044B13B10448AFF337
S3150800011C00800123237010BD100000200000000091
S3150800012C0817000808B5034B1BB103490348AFF37E
S3150800013C008008BD00000000140000200817000805
S3150800014C72B6704762B6704708B5FFF7F9FF08BD77
S3150800015C10B500F0CDF900B910BD00F07FFD0028F0
S3150800016CFAD000F047FB00F0D7F900F0C3FD00F019
S3150800017CC3F920F0604020F07F00044B986000F033
S3150800018CBBF94468FFF7DEFFA047E5E700ED00E0A2
S3150800019C70B508E0461C4D1C0B78037000F05EFB2E
S315080001AC304629462246531E9CB2002AF2D170BD0F
S315080001BC08B5C1F3080353B90368994209D040F846
S315080001CC041B4FF40072FFF7E3FF012008BD002063
S315080001DC08BD012008BD2DE9F041074600F074FE64
S315080001EC00247F2C14D83E68A30006EB03083B4476
S315080001FC5D6800F033FB2A4600234146022000F0D6
S3150800020CBDFE38B956F824309D4209D10134E8E7C9
S3150800021C012400E0002400F071FE2046BDE8F081C0
S3150800022C0024F8E738B50D460B4B984208D004461F
S3150800023C0A4B994206D0FFF7CEFF20B9002407E0F7
S3150800024C074C00E0044C29462046FFF7B1FF08B1DD
S3150800025C204638BD0024FBE73002002000200008A9
S3150800026C2C0000202DE9F04106460C4617461D4683
S3150800027C21F4FF7828F001080368B3F1FF3F0DD08D
S3150800028C3368984505D041463046FFF7CBFF0646FE
S3150800029C28B33368E41A344404340CE04146FFF7B7
S315080002AC87FF03460028EBD116E017F8013B04F844
S315080002BC013B013D0FD000F0D1FA331DE31AB3F51B
S315080002CC007FF2D308F500713046FFF7ABFF064600
S315080002DC38B1041DE9E701231846BDE8F08100236F
S315080002ECFAE70023F8E700004FF0FF33024A1360E1
S315080002FC024A1360704700BF2C0000203002002011
S3150800030C10B54B1E114C241AA34218D8104B984200
S3150800031C17D90B18013B0D4CA34214D80B460146B2
S3150800032C20F4FF7020F001000A4CA04203D00A48C2
S3150800033CFFF798FF10BD0948FFF794FF10BD002082
S3150800034C10BD002010BD002010BD00BFFFFF010826
S3150800035CFF1F0008002000082C0000203002002097
S3150800036C30B587B0002305934A1E1F4B1B1A9A42B9
S3150800037C31D820F47F7323F003031C4A93422ED9F9
S3150800038C0A18013A184CA2422BD8C01A0144C1F3D8
S3150800039C8F25C1F3090109B10135ADB200240194C9
S315080003AC03930123049300F08FFDA5420DD900F0A9
S315080003BC55FA05A901A800F053FE50B9039B03F59D
S315080003CC806303930134A4B2EFE7012400F096FD91
S315080003DC02E00024FAE70024204607B030BD0024CA
S315080003ECFAE70024F8E700BFFFFF0108FF1F000823
S315080003FC104B1B68B3F1FF3F1AD000B583B00D4AFA
S3150800040C536891680B44D1680B4411690B445169C4
S3150800041C0B4491690B44D26913445B4202AA42F815
S3150800042C043D04210448FFF76BFF03B05DF804FB99
S3150800043C01207047300200200C2100080D4B1B6868
S3150800044C0D4A126813440D4A126813440C4A126872
S3150800045C13440C4A126813440B4A126813440B4A89
S3150800046C126813440A4A1268D34201D00020704716
S3150800047C0120704700200008042000080820000806
S3150800048C0C2000081020000814200008182000086A
S3150800049C0C21000808B50C4B1B68B3F1FF3F04D0C0
S315080004AC0948FFF798FE034650B1084B1B68B3F191
S315080004BCFF3F07D00548FFF78EFE034600B1012320
S315080004CC184608BD0123FBE7300200202C0000204B
S315080004DC004870470020000808B5FFF705FF08BD5F
S315080004EC08B5FFF70DFF08BD08B5FFF739FF08BDBE
S315080004FC08B5FFF7A3FF08BD08B5FFF7E9FF08BD68
S3150800050C08B5FFF775FF034608B9184608BDFFF787
S3150800051CC1FF0346F9E700000022014B1A60704739
S3150800052C10E000E008B5FFF7F7FF054B054A5A60DF
S3150800053C00229A6005211960034B1A6008BD00BF9A
S3150800054C10E000E03F19010034040020044B1B683E
S3150800055C13F4803F03D0034A1368013313607047C2
S3150800056C10E000E03404002008B5FFF7EFFF014B5C
S3150800057C186808BD3404002008B5FFF7F5FF08BD58
S3150800058C70470000054B1B6813F0200F04D0034B73
S3150800059C5B680370012070470020704700440040D8
S315080005AC10B5094B5860FFF7DFFF00F10A04064B3C
S315080005BC1B6813F0800F05D100F050F9FFF7D4FF34
S315080005CC8442F4D210BD00BF0044004010B586B07A
S315080005DC4FF46143009300230193029303930C2277
S315080005EC04920593094C6946204600F0BFFE236920
S315080005FC23F490432361636923F02A036361E36858
S3150800060C43F40053E36006B010BD00BF004400403D
S3150800061C70B506460D46402904D82846FFF7C0FF94
S3150800062C00240BE06F21074800F064F8F5E700F0AA
S3150800063C15F9305DFFF7B4FF0134A4B2ABB29C4296
S3150800064CF5D370BD2017000870B5254B1C78BCB9BE
S3150800065C2448FFF797FF012801D0204670BD214B8F
S3150800066C1B78013BDBB23F2BF7D8FFF77DFF1E4B00
S3150800067C186000221D4B1A700122194B1A70ECE7F0
S3150800068C06460D46194B1B78013316481844FFF7D6
S3150800069C79FF044601280AD0FFF766FF124B1B6840
S315080006AC6433984219D900240D4B1C70D5E70F4BAF
S315080006BC1A780132D2B21A700A4B1B789A4201D0B8
S315080006CC0024CAE70A493046FFF762FD0022044BAC
S315080006DC1A70064B1B782B70BFE70024BDE700BFCA
S315080006EC79040020380400207C0400207A040020B9
S315080006FC3904002008B500F0B1F8FCE708B500F09D
S3150800070CA1F8012803D00B4B1B78012B00D008BD90
S3150800071CFFF72AFF084B1B68084A1268134403F5AF
S3150800072CFA739842F3D30022024B1A70FFF710FDA6
S3150800073CEDE700BF84040020800400208804002014
S3150800074C08B5054B1B78012B00D008BDFFF70CFF2D
S3150800075C024B1860F9E700BF8404002088040020C7
S3150800076C08B50122034B1A70FFF7EAFFFFF7C6FF1D
S3150800077C08BD00BF8404002008B5FFF7E5FC00F0AF
S3150800078C69F8FFF7CFFEFFF7A7FE00F00DF8FFF7A5
S3150800079CE7FF08BD08B500F061F8FFF7D7FE00F0D3
S315080007AC0FF8FFF7ABFF08BD08B500F0C5F9FFF762
S315080007BC0DFF0022014B1A7008BD00BF0000002077
S315080007CC00B583B00DF107010848FFF73DFF012876
S315080007DC02D003B05DF804FB0022054B1A709DF895
S315080007EC0710024800F0C8F9F3E700BF8C04002094
S315080007FC000000207047000008B5054B1B7813B1A4
S3150800080C00F0B2F908BDC9B2FFF702FFF8E700BF5E
S3150800081C00000020044B1B78013B022B01D9402019
S3150800082C70470020704700BF00000020044B1B785F
S3150800083C013B022B01D9402070470020704700BFAE
S3150800084C0000002008B500F085F9034600B1012325
S3150800085C184608BD08B500F00FFA08BD08B500F033
S3150800086C10FA08BD0022014B5A707047CC040020C0
S3150800087C034BFE22DA7018710222A3F84420704743
S3150800088CCC04002010B5054C00232370FFF7EAFFB3
S3150800089CFF23E3700123A4F8443010BDCC040020D8
S315080008AC064BFF22DA7000221A71597859719A711F
S315080008BCDA711A720622A3F844207047CC04002079
S315080008CC08B50020FFF7D4FF08BD0000074BFF2230
S315080008DCDA70074A9A6400221A715A719A710722B9
S315080008ECC3F807200822A3F844207047CC0400203C
S315080008FC4C170008044BFF22DA7042689A640122EE
S3150800090CA3F84420704700BFCC04002008B531205A
S3150800091CFFF7AEFF08BD000038B5084CFF23E3709F
S3150800092C002525716571FFF775FFA071E5712572B4
S3150800093C65720723A4F8443038BD00BFCC040020E8
S3150800094C38B5FFF78FFF0E4C01252570FF23E37092
S3150800095C1023237100236371FFF75CFFA071FFF767
S3150800096C65FFE071FFF762FFC0F30720207265721E
S3150800097CA5720823A4F84430FFF7AEFD38BD00BFB6
S3150800098CCC04002038B505464478FFF743FF0138F8
S3150800099C844210DC0A4C6A78A16C201DFFF7F8FB20
S315080009ACFF23E3706A78A36C1344A3646B78013352
S315080009BCA4F8443038BD2220FFF75AFF38BD00BFD3
S315080009CCCC04002038B504464578FFF723FF0138D8
S315080009DC854211DC61680A4DA9646278281DFFF707
S315080009ECD7FBFF23EB706278AB6C1344AB6463786C
S315080009FC0133A5F8443038BD2220FFF739FF38BD3E
S31508000A0CCC040020F8B505461746002406E015F870
S31508000A1C013B1C44E4B2FFF721FF31464E1E002968
S31508000A2CF5D13C600120F8BD10B5084CFF23E370E6
S31508000A3CE21D4168A06CFFF7E5FF20710023637186
S31508000A4CA3710823A4F8443010BD00BFCC040020C1
S31508000A5C38B505460D4B9C6CFFF7DCFE6A1C411E2F
S31508000A6C2046FFF73DFD60B1084CFF23E370FFF706
S31508000A7CD1FE0138A36C0344A3640123A4F84430C3
S31508000A8C38BD3120FFF7F4FE38BD00BFCC0400207A
S31508000A9C38B504464578FFF7BDFE023885420EDCAC
S31508000AAC114BFF22DA700122A3F84420617851B960
S31508000ABCFFF726FD90B93120FFF7DAFE38BD222064
S31508000ACCFFF7D6FE38BDA21C074B986CFFF708FD3E
S31508000ADC28B16178044A936C0B44936438BD312071
S31508000AECFFF7C6FE38BD00BFCC04002008B5416828
S31508000AFC074B986CFFF7F8FC30B1054BFF22DA7000
S31508000B0C0122A3F8442008BD3120FFF7B1FE08BD29
S31508000B1CCC04002008B5FFF71BFB034BFF22DA7049
S31508000B2C0122A3F8442008BDCC04002008B589B2DC
S31508000B3CFFF762FE08BD0000054B00221A709A6486
S31508000B4C83F84320A3F844209A705A70704700BF64
S31508000B5CCC040020034B1B780BB1012070470020F6
S31508000B6C704700BFCC0400200022024B83F84320B8
S31508000B7C704700BFCC04002008B50378FF2B04D0BF
S31508000B8C354A1278012A14D008BDFFF7D9FE324B24
S31508000B9C93F84330012B5AD02F4BB3F94410002944
S31508000BACF2DD1846012380F843300330FFF7BEFF09
S31508000BBCEAE7C93B352B46D8DFE803F0334545420F
S31508000BCC45453F363C3945454545454545454545E5
S31508000BDC45454545454545454545454545454545AB
S31508000BEC454545454545241E1B2145454527452A6A
S31508000BFC2D30FFF7C7FECAE7FFF7E4FEC7E7FFF796
S31508000C0C79FEC4E7FFF710FFC1E7FFF75FFEBEE703
S31508000C1CFFF756FEBBE7FFF743FEB8E7FFF732FED2
S31508000C2CB5E7FFF715FFB2E7FFF732FFAFE7FFF7B8
S31508000C3C73FEACE7FFF75AFFA9E7FFF76BFFA6E7CA
S31508000C4CFFF764FEA3E72020FFF712FE9FE71020AC
S31508000C5CFFF70EFEA0E700BFCC04002008B5054B35
S31508000C6C9B6813F4005F01D1002008BD00F03CF826
S31508000C7C012008BD0010014008B5642000F006F8F4
S31508000C8C08BD08B500F008F808BD0000014B18802F
S31508000C9C704700BF1805002008B5FFF765FC0E4B1A
S31508000CAC1B6898420FD30D4B1B786BB901220B4B63
S31508000CBC1A7020220A4B1A61FFF756FC094B1B883F
S31508000CCC1844054B186008BD0022044B1A702022E4
S31508000CDC034B5A61F0E700BF1C0500201A050020DB
S31508000CEC00080140180500202022014B5A61704764
S31508000CFC0008014010B5064B4FF0FF32DA600024AD
S31508000D0C1C61DA60DC6000F08BFC204610BD00BF6D
S31508000D1C0010024010B504460E4B18784FF47A733F
S31508000D2CB3FBF0F30C4A1068B0FBF3F000F06EF866
S31508000D3C68B90F2C01D9012010BD002221464FF0AD
S31508000D4CFF3000F031F8054B1C60002010BD012067
S31508000D5C10BD00BF01000020080000200400002080
S31508000D6C08B5074A136843F010031360032000F014
S31508000D7C09F80020FFF7CEFF00F0EEFB002008BDB7
S31508000D8C00200240074AD36823F4E0631B041B0CBB
S31508000D9C000200F4E060184340F0BF6040F40030F5
S31508000DACD060704700ED00E030B4164BDB68C3F337
S31508000DBC0223C3F10704042C28BF04241D1D062D89
S31508000DCC17D9033B012505FA04F4013C2140994047
S31508000DDC05FA03F3013B1340194300280BDB090101
S31508000DECC9B200F1604000F5614080F8001330BCD0
S31508000DFC70470023E6E700F00F000901C9B2024B61
S31508000E0C1954F4E700ED00E014ED00E00138B0F1F8
S31508000E1C807F0AD2064B5860F021064A82F82310C6
S31508000E2C0020986007221A6070470120704700BF9F
S31508000E3C10E000E000ED00E00022044BDA61044A01
S31508000E4C136943F0010313610180704720050020E4
S31508000E5C002002401A4BDB6813F0100F27D0194AF2
S31508000E6CD36943F00203D3611023154AD26812F0F2
S31508000E7C040F06D01349CA6942F00102CA6143F04D
S31508000E8C04030F4AD26912F0010F09D00D49CA6939
S31508000E9C42F00402CA610A49CA6922F00102CA610F
S31508000EAC40F20112934204D0054AD36070470023DE
S31508000EBCDBE7034AD36923F00103D361704700BF0C
S31508000ECC00200240200500200A4B1B6913F0800FF6
S31508000EDC0DD0084B084A5A6002F188325A601B69D1
S31508000EEC13F0800F01D001207047002070470020B6
S31508000EFC704700BF0020024023016745034A136967
S31508000F0C43F0800313610020704700BF00200240A5
S31508000F1C38B50446FFF730FB0546174BDB6813F06C
S31508000F2C010F0AD0B4F1FF3FF7D00CB3FFF724FB3F
S31508000F3C401B8442F1D2032038BD0F4BDB6813F0FB
S31508000F4C200F02D020220C4BDA600B4BDB6813F017
S31508000F5C100F09D1084BDB6913F0010F04D1064BAE
S31508000F6CDB6813F0040F05D0FFF774FF012038BDBA
S31508000F7C032038BD002038BD002002402DE9F84377
S31508000F8C234C247E012C03D102231846BDE8F88392
S31508000F9C1E4690460F46044601221D4B1A764CF205
S31508000FAC5030FFF7B5FF034670BB012C29D0022C35
S31508000FBC24D04FF0040900244C4525D22101C1F157
S31508000FCC2002A1F1200328FA01F106FA02F21143D4
S31508000FDC26FA03F3194389B207EB4400FFF72CFFF3
S31508000FEC4CF25030FFF794FF0A4B1D6925F00105AA
S31508000FFC1D61034640B90134E4B2DDE74FF002093E
S3150800100CD9E74FF00109D6E70021014A1176BCE76A
S3150800101C20050020002002400022064BDA61064B10
S3150800102C1A6942F004021A611A6942F040021A61FE
S3150800103C704700BF20050020002002400022064B06
S3150800104CDA61064B1A6942F002021A6158611A698A
S3150800105C42F040021A617047200500200020024029
S3150800106C264B1B7E012B46D070B50E460546012233
S3150800107C224B1A760368022B20D04CF25030FFF71D
S3150800108C47FF90BB4FF0FF333360AC680121EA6829
S3150800109CAB6803EB82239C4228D22046FFF7CEFF8F
S315080010AC4CF25030FFF734FF154A136923F002034C
S315080010BC13610146B8B904F58064E8E74CF2503080
S315080010CCFFF726FF08B1012110E00120FFF7A4FF66
S315080010DC4CF25030FFF71CFF0146094A136923F0FE
S315080010EC0403136102E0346000E001210022034B83
S315080010FC1A76084670BD022108467047200500205E
S3150800110C00200240264B98420DD0264B984216D00A
S3150800111C254B98421FD0254B984228D0244B9842F1
S3150800112C31D00020704703F58433DA6842F00402A4
S3150800113CDA60DA6822F00402DA600120704703F5F7
S3150800114C8233DA6842F00802DA60DA6822F00802BA
S3150800115CDA600120704703F58033DA6842F0100232
S3150800116CDA60DA6822F01002DA600120704703F5BB
S3150800117C7C43DA6842F02002DA60DA6822F0200250
S3150800118CDA600120704703F57843DA6842F04002CA
S3150800119CDA60DA6822F04002DA600120704700BF94
S315080011AC00080140000C01400010014000140140E9
S315080011BC00180140F0B50D68C5F30F2595FAA5F290
S315080011CCB2FA82F233E0A2F108044FF00113A340FD
S315080011DC43F080634E681F0EC45993FAA3FEBEFAF9
S315080011EC8EFE4FEA8E0E4FF00F0C0CFA0EFE24EA0A
S315080011FC0E0493FAA3FEBEFA8EFE4FEA8E0E06FA7C
S3150800120C0EF63443C451C6681C0A26EA040E94FA30
S3150800121CA4F4B4FA84F40E6906FA04F44EEA040447
S3150800122CC4604C68012C0FD0092C0DD0013235FA4C
S3150800123C02F337D0012393401D42F7D0072AC2D8B0
S3150800124C40F201139340C5E7C45993FAA3F6B6FACC
S3150800125C86F6B6004FF0030E0EFA06F624EA060ECC
S3150800126C93FAA3F6B6FA86F6B6008C6804FA06F66E
S3150800127C46EA0E06C651CC6893FAA3FEBEFA8EFE53
S3150800128C4FEA8E0E4FF0040C0CFA0EFE26EA0E06EA
S3150800129C93FAA3F3B3FA83F39B0004FA03F33343E9
S315080012ACC351C3E70120F0BD034B5B68C3F30313BB
S315080012BC024AD35CD8407047001002405417000805
S315080012CC034B5B68C3F30223024AD35CD8407047CE
S315080012DC0010024064170008034B5B68C3F3C22373
S315080012EC024AD35CD84070470010024064170008C5
S315080012FC0B4B5B6803F480337BB1094B586800F4DD
S3150800130C00300130074BB3FBF0F0054B5B68C3F3B9
S3150800131C8343023303FB00F070470348F5E700BF2D
S3150800132C0010024000127A0000093D0008B5054B72
S3150800133C5B6803F00C03082B02D1FFF7D9FF08BD35
S3150800134C014808BD0010024000127A0010B5044688
S3150800135CFFF7ECFF2060FFF7A7FF6060FFF7B0FF11
S3150800136CA0606068FFF7B8FFE06010BDC36813F4AF
S3150800137C005F01D00020704770B584B00D46044656
S3150800138CC36823F4B05323F00C034A68C9680A43AC
S3150800139C29690A431343C360AB68026922F44052B5
S315080013AC134303616B69426922F440721343436128
S315080013BC6846FFF7CBFF1C4B9C422AD01B4B9C4222
S315080013CC29D01B4B9C4228D0002343B3296849B328
S315080013DC03EB830303EB83038900B3FBF1F1154E8F
S315080013ECA6FB01356D092A0190B2642202FB15127F
S315080013FC13013233A6FB0323C3F34F1303F0F00296
S3150800140C024492B203F00F0313449BB2A36001206B
S3150800141C06E0039BD9E7029BD7E7029BD5E700209A
S3150800142C04B070BD0020FBE70038014000440040C2
S3150800143C004800401F85EB51014B1860704700BFF0
S3150800144C080000200F4B1A6842F001021A6059680E
S3150800145C0D4A0A405A601A6822F0847222F48032C5
S3150800146C1A601A6822F480221A605A6822F4FE025C
S3150800147C5A604FF41F029A604FF00062034B9A6051
S3150800148C704700BF001002400000FFF800ED00E0B6
S3150800149C08B5264A136823F0070343F002031360C2
S315080014AC136803F00703022B03D068212048FFF7C3
S315080014BC21F9204B1A6842F480221A601A6842F401
S315080014CC80321A601B4B1B6813F4003FFAD0194A7A
S315080014DC536823F47C1343F4E8135360136843F0FE
S315080014EC80731360134B1B6813F0007FFAD0114BF3
S315080014FC5A6822F0F0025A605A6822F4E06242F402
S3150800150C80625A605A6822F460525A605A6822F00D
S3150800151C030242F002025A60064B5B6803F00C03A6
S3150800152C082BF9D10448FFF787FF08BD00200240B5
S3150800153C6C1700080010024000A24A0408B5FFF711
S3150800154C0FFCFFF7A5FF08BD08B5FFF7F7FFFFF778
S3150800155C13F9FFF71FF9FCE7F0B58BB02D4B9A6919
S3150800156C42F001029A619A6902F001020492049A05
S3150800157CDA6942F08052DA61DA6902F08052039233
S3150800158C039A9A6942F004029A619A6902F0040273
S3150800159C0292029A9A6942F010029A619A6902F0CA
S315080015AC10020192019ADA6942F40032DA61DB69B7
S315080015BC03F400330093009B42F2200305930123A6
S315080015CC06930227079700260896134C05A920466A
S315080015DCFFF7F0FD2023636103F18463059304236D
S315080015EC069305A90D48FFF7E5FD40F2044305935C
S315080015FC092506950797089605A92046FFF7DAFDEB
S3150800160C40F608030593069505A92046FFF7D2FD73
S3150800161C0BB0F0BD0010024000080140001001405C
S3150800162C08B50E48FFF76EFD0D48FFF76BFD0D4B21
S3150800163CDA6922F40032DA619A6922F010029A61A8
S3150800164C9A6922F004029A61DA6922F08052DA6108
S3150800165C9A6922F001029A6108BD00BF0010014088
S3150800166C0008014000100240002103E00B4B5B58B8
S3150800167C435004310A480B4B42189A42F6D30A4A8D
S3150800168C02E0002342F8043B084B9A42F9D3FFF7D1
S3150800169CD9FE00F00FF8FFF757FF704780170008C0
S315080016AC000000200C00002010000020400500203F
S315080016BCFEE7000070B500250C4E0D4CA41BA410BB
S315080016CCA54209D100F01AF800250A4E0A4CA41BAB
S315080016DCA410A54205D170BD56F82530984701359A
S315080016ECEEE756F8253098470135F2E778170008E3
S315080016FC78170008781700087C170008F8B500BF9B
S3150800170CF8BC08BC9E467047F8B500BFF8BC08BCC8
S3090800171C9E46704720
S315080017202E2E5C2E2E5C2E2E5C2E2E5C536F757222
S3150800173063655C41524D434D335F53544D333246D6
S31508001740315C756172742E63000000004F70656E1F
S31508001750424C54000000000000000000010203048F
S315080017600607080900000000010203042E2E5C6D1E
S30D0800177061696E2E630000009A
S309080017783101000825
S3090800177C0D01000845
S31108001780040100001000000000A24A044A
S7050800167567
